:0831A80033302E3220202000FC
:082DFA00C102C108C100C109BA
:0331E800C2B4224C
:0331EB00D2B42239
:0D30E000A2B4E43370047F0180027F00225F
:102DD80075A40D7580FF75D44075A50C75F20F7537
:102DE800D50175F3F075A63075B0FF75E10675E28B
:022DF800C222F5
:1030C10075BC4475E8C075BA1F75D10843E608227E
:0C313B0075A14075F80975A202D2AE2201
:0431E40075B283221B
:0A31800075DA2175DB2143E6102209
:0D30ED007592077593F875910443E68022F3
:0B1A070075CA3475CBFFD2CAD2AD22E5
:10304A00758850758922758E0C758AAE758CAE7529
:06305A008BC7758DC72233
:102F1C00E4F5D91231E4122DD81230C112313B1222
:0B2F2C003180121A071230ED02304A0B
:10307600E4FEEF139293C292D292EFC313FF0EEEC9
:03308600B408EF9C
:013089002224
:102B0600752CFFE55014600F146011146013240334
:102B1600700F532C7F800A532CBF8005532CDF8007
:102B260000E55114600F1460111460132403700F34
:102B3600532CEF800A532CF78005532CFB8000E5BD
:0B2B46004F6003532CFCAF2C023076D4
:0D30FA00754200754301854B2E854C2F2239
:0D310700754400754501854D30854E31221F
:0C314700E4F542F543853A2E853B2F222B
:0C315300E4F544F545853C30853D312213
:10306000E54F6005E4F528F529752600752701125E
:0630700030FA752B01226D
:0D311400752800752901123107752B022264
:10308A00C203C205E4F547F548F526F527F52E757E
:03309A002F0122E1
:10309D00C204C207E4F549F54AF528F529F530755E
:0330AD00310122CC
:061A1B0012308A02309D2A
:102FEB0075BB1175E8D030EDFDC2EDE5BED394C0D5
:082FFB004003D20B22C20B229D
:102FB900121A1BE54F6003023060E55070031230AE
:092FC90060E5517003123114227D
:0F30D1009002DEE0C3941E5005EFF01231DE22B4
:052F37009002DEE0FF46
:102F3C009002DEE0C3941E500BEFF0122CF8122F0F
:052F4C00B9122B062262
:102A5B00E4FF75BB12FE75E8D030EDFD74252EF545
:102A6B0082E43403F583E5BEF00E05BBEEC394029E
:102A7B0040E4900325E0FED394194021A3E0FDD35D
:102A8B0094194019EE94CC5004C2148002D214ED68
:102A9B00C394CC5004C2158008D2158004C215C251
:0E2AAB0014A214E43325E0FFA215E4334FFF1C
:012AB90022FA
:102B5100EF25E0FFA20BE4334FFFB408005037909C
:102B61002B67F8282873022B7F022B82022B850208
:102B71002B88022B8B022B8E022B91022B947F38F8
:102B8100227F39227F3A227F3B227F3C227F3D22D6
:092B91007F3E227F3F227F3822A3
:100EAA00122F1C122A5B900264EFF075460F753AF6
:100EBA0000753B01754B00754C01753C00753D0191
:100ECA00754D00754E01121A1BC2A4C2A5750807FA
:100EDA007509D0122FEBE0FF122B51900304EFF0AB
:100EEA0012312E43F601300B031231EBD2AF12301E
:100EFA001B122CF8122FB9122B063008081231DEF9
:100F0A001231EBC208300010900304E0FF7BFF7A35
:100F1A003179A81229FBC20030090A900304E0FFC4
:100F2A00122E3EC209E525606C14604D24FD603422
:100F3A0024FC601E24067057634F01121A1BE54FEA
:100F4A007004E5507003123060E5517027123114B5
:100F5A0080220550E550B40403E4F55012308A1299
:100F6A00306080100551E551B40403E4F5511230A4
:100F7A009D123114122FD28016300213300B101228
:100F8A0030E0EF60051231EB80051231E8C216122B
:0B0F9A002B06E4F525200103021106E0
:100FA500C201E50945086008E5091509700215083B
:100FB5007D04E4FF1213357D057F011213357D068F
:100FC5007F021213357D077F03121335E552251372
:100FD500FEE433900281F0A3CEF0C2AD900281E031
:100FE500FEA3E0FF9008A875F003121D5DEE75F0F5
:100FF50003A42583F583E493F53E740193F53F90AF
:1010050008A775F003EF121D5DEE75F003A42583A7
:10101500F583E493754B00F54CD2ADE5542512FEEE
:10102500E433900281F0A3CEF0C2AD900281E0FEE0
:10103500A3E0FF9008A875F003121D5DEE75F0039F
:10104500A42583F583E493F532740193F533900871
:10105500A775F003EF121D5DEE75F003A42583F56A
:1010650083E493753A00F53BD2ADE5532514FEE4D0
:1010750033900281F0A3CEF0C2AD900281E0FEA3D1
:10108500E0FF9008A875F003121D5DEE75F003A44E
:101095002583F583E493F540740193F5419008A702
:1010A50075F003EF121D5DEE75F003A42583F5833E
:1010B500E493754D00F54ED2ADE5552515FFE433A6
:1010C500FE900281F0A3EFF0C2AD9008A875F00381
:1010D500121D5DEE75F003A42583F583E493F534C5
:1010E500740193F5359008A775F003EF121D5DEEB9
:1010F50075F003A42583F583E493753C00F53DD293
:01110500AD3C
:101106007B017A027965122CCCEF7003020F0490F2
:101116000267E0121D6911920411D90511541411C8
:101126003B1611481711591A117B1B11861D118C7C
:101136001E00001229300B051231E8C216D2020237
:101146001229200B030212291231EB021229D202B4
:101156000212297B017A027965900275EBF0A3EA07
:10116600F0A3E9F0121B26FE900304E0FF6E600375
:101176000212298005900304E0FF122E5F02122955
:101186001231BF0212291231D80212297B017A02CA
:101196007965900278EBF0A3EAF0A3E9F0900003FA
:1011A600121B3FFF900304E06F707820B46D90022D
:1011B6007804F0A3EAF0A3E9F0900005121B3FFFC4
:1011C600900006121B3FFD900004121B3FFB1227E6
:1011D6007080487B017A027965900278EBF0A3EA89
:1011E600F0A3E9F0900003121B3FFF900304E06FA9
:1011F600703120B42690027804F0A3EAF0A3E9F057
:10120600900005121B3FFF900006121B3FFD900049
:1012160004121B3FFB122553122F37900304E0FFE5
:10122600122EC130B403020F04200203020F0490F1
:101236000267E014603924FA60561470030212E063
:1012460024F97003021315240D6003020F041230F3
:10125600B07B017A027965900275EBF0A3EAF0A300
:10126600E9F0900003121B3FFF1230D102130F1258
:1012760030B07B017A027965900275EBF0A3EAF053
:10128600A3E9F0900003121B3FFF122F3C02130F3D
:101296001230B07B017A02796590027BEBF0A3EA0B
:1012A600F0A3E9F0900003121B3FFF900004121B0D
:1012B6003FFD900005121B3FFBC00390027BE0FB45
:1012C600A3E0FAA3E0F9900006121B3F900286F015
:1012D600D0031226BE122F37802F1230B07B017A30
:1012E60002796590027BEBF0A3EAF0A3E9F09000A7
:1012F60003121B3FFF900004121B3FFD90000512D6
:101306001B3FFB121F5C122F37123194020F049001
:101316000264E06003020F047B017A0279659002A1
:0F1326007E04F0A3EAF0A3E9F012246B020F0497
:10260900E5B0540FF5246546600CE5246546F52AC6
:10261900752D03852446E52D6052152DE52D704C49
:10262900E52A30E11DE52420E11890030230020972
:102639007405F0A374DCF080077401F0A37477F0DB
:10264900D206E52A30E308E52420E303752508E5E9
:102659002A30E208E52420E203752504300B0DE554
:102669002A30E008E52420E00375250130062E9084
:102679000303E024FFF0900302E034FFF0E5B054D7
:10268900026005752502C206900302E07002A3E00C
:10269900700BC206300204D2008002D208E5394527
:1026A900386011E539153970021538144538700448
:0426B900D2A6D2A72C
:0126BD0022FA
:0331EE00D2FA22F0
:102EE000E549C4F854F0C8E54AC4540F48F5A39026
:0E2EF00002FF74FFF0A37431F0A374EEF02221
:102F5100C2FAE549C4540F44A0F5A39002FF74FFDF
:0A2F6100F0A3742EF0A374E0F02238
:0331F100D2FA22ED
:102EFE00E547C4F854F0C8E548C4540F48F5A3900C
:0E2F0E0002FF74FFF0A37431F0A374F1F022FF
:102F6B00C2FAE547C4540F4490F5A39002FF74FFD7
:0A2F7B00F0A3742EF0A374FEF02200
:031A1500022B9A07
:102B9A00C0E0C0F0C083C082C0D075D000C000C001
:102BAA0001C002C003C004C005C006C007C2FF902E
:102BBA0002FFA3E0FAA3E0F9121D8FD007D006D0D6
:102BCA0005D004D003D002D001D000D0D0D082D01A
:062BDA0083D0F0D0E032D0
:061A2700D2A47536032273
:0631C600D2A575370322BB
:031A120002172C8C
:10172C00C0E0C0F0C083C082C0D075D000C000C083
:10173C0001C002C003C004C005C006C007C2CF2050
:10174C000A03021804C20AE5366005D53602C2A4A3
:10175C00E527452670030217F3E52F152F700215A8
:10176C002E14452E60030217F3E5436401454270C5
:10177C003D854B2E854C2FE550B402062086033058
:10178C000306122991EF605FE54F6008E52BB40169
:10179C0003123114E54F6006E52B64037049E550E4
:1017AC00B4020620864120033E12314780391231A3
:1017BC00471229ABEF6030E54F600AE52BB4030FFD
:1017CC00752B048007300504C2058003121A27E527
:1017DC004F6005E52BB4010FE550700512306080A9
:1017EC00067526007527009002FF74FFF0A3742F76
:1017FC00F0A3746BF00218ABD20AE5376005D5374D
:10180C0002C2A5E5294528700302189DE531153162
:10181C00700215301445307078E54564014544700C
:10182C0041854D30854E31E54F700BE551B40206C4
:10183C002090033004061229C6EF6055E54F60086E
:10184C00E52BB40203752B03E54F6006E52B64040E
:10185C00703FE551B4020620903720043412315306
:10186C00802F1231531229E0EF6026123107300716
:10187C0004C20780031231C6E54F6007E5507003C0
:10188C00123060E54F7004E551600675280075292B
:10189C00009002FF74FFF0A3742FF0A37451F0D2E8
:1018AC00FFD007D006D005D004D003D002D001D091
:0C18BC0000D0D0D082D083D0F0D0E03239
:031A2D00022D91F6
:102D9100C0E0C083C082C0D075D000C00753917F0E
:102DA10012260975BB0475E8D0D007D0D0D082D0E7
:042DB10083D0E032B9
:031A2100022C9FF5
:102C9F00C0E0C0D075D000C000C007C2EDAFBB749C
:102CAF000E2FF8A6BEE5BB640B600705BB75E8D019
:0D2CBF008002D201D007D000D0D0D0E0328A
:031A2400022D4749
:102D4700C0E030D80BC2D8E550640360031230608E
:102D570030D90FC2D9E54F7009E5516403600312FA
:052D67003114D0E03240
:10299100E548253FF548E547353EF54740037F00CB
:1029A100227F0174FFF547F54822C3E5489533F5C9
:1029B10048E5479532F54740037F00227F017400C7
:1029C100F547F54822E54A2541F54AE5493540F5FF
:1029D1004940037F00227F0174FFF549F54A22C374
:1029E100E54A9535F54AE5499534F54940037F00B7
:0A29F100227F017400F549F54A2227
:102E0200420262000042020D00004202080000C1BC
:052E120013C112C11103
:0A318A00C212C213E490020CF022FE
:102DB500E4900262F0A3F090020DF0A3F0A3F0906E
:102DC5000208F0A3F0900203F0A37440F0E490022F
:032DD5000BF022DE
:0631CC0012318A022DB54C
:0D31210075C19043E60190020A7401F0228E
:1030B00043C140E5C120E5FB1231CCE490020AF0A7
:0130C00022ED
:0A31940053C1BF90020A7401F0223B
:0D312E00AE07123121900207EEF00231CC05
:102D6C00E4900343F0A3F0301202FF222013FDD2B3
:102D7C0012900205E4F0A37410F0900250EFF0E40E
:042D8C00A3F07F0130
:012D90002220
:1019D30030120A900205E07002A3E070037F002238
:1019E300900206E024FFF0900205E034FFF090023D
:1019F30051E0FE04F074522EF582E43402F583EFD5
:041A0300F07F01224D
:0B315F00301207C212D21312319E2260
:0A319E00E5C120E5FBC2C4D2C52242
:10291800900307EBF0A3EAF0A3E9F090020AE07055
:1029280002FF2290030AE0FE6005D3941040037F63
:082938000022122D6CEF604E2D
:10294000E490030CF090030AE0FF90030CE0FEC358
:102950009F5024900307E0FBA3E0FAA3E0F98E82E6
:10296000758300121B3FFF1219D3EF7002FF2290F4
:10297000030CE004F080CEE490020CF012315F9082
:0E298000030BE070032013FD90020CE0FF2219
:03298E007FFF22A6
:0E18C800900329EBF0A3EAF0A3E9F0A3EDF002
:1018D600E4FFD3900263E09400900262E064809497
:1018E6008050012253E6FE900208E0FEA3E0240F9A
:1018F600F58274023EF583E0FF900208E475F0017C
:10190600121BA0FCE5F064404C7006900208F0A3A0
:10191600F0900204E004F07006900203E004F0E4A4
:10192600FE90032CE0FDEEC39D5054EEC39F504F36
:10193600900208E0FCA3E0240FF58274023CF583D4
:10194600E0FD900329E0FBA3E0FAA3E0F98E82759F
:101956008300ED121B7E900208E475F001121BA0B5
:10196600FCE5F064404C7006900208F0A3F090028B
:1019760004E004F07006900203E004F00E80A2EE8C
:10198600C39F5029900208E475F001121BA0FCE5E4
:10199600F064404C7006900208F0A3F0900204E058
:1019A60004F07006900203E004F00E80D290026309
:1019B600E024FFF0900262E034FFF043E60190037A
:0C19C6002CE0FEEFC39E50028002AF0632
:0119D20022F2
:10300300D3900263E09400900262E0648094804075
:08301300047F0180027F00220E
:031A1800021DC1EB
:101DC100C0E0C0F0C083C082C0D075D000C000C0E8
:031DD10006C00742
:101DD400C218E5C054FE121D691EB0081EB00A1ECA
:101DE400770C1E770E1F29101F29121E7D221E88B4
:101DF400281E882A1E7D2C1E7D2E1E6AC01E23C20C
:101E04001E0EE01E0EE200001F34C211900250E0CC
:101E1400F5C2C2C5C2C490024F74FFF0021F3690CF
:101E2400024FE0FFB4FF12900251E0F5C2C2C5C2F6
:101E3400C490024FE4F0021F36900251E0FEEFC35B
:101E44009E501790024FE0FF04F074522FF582E485
:101E54003402F583E0F5C2021F36D2C490020CE4CA
:101E6400F0C213021F3690020C74FDF0D2C5C2C436
:101E7400021F3690024F74FFF0D211C2C4C2C1D205
:101E8400C5021F36E5C26007900207E0B5C20E9096
:101E94000202E4F0C2C5C2C4D2C1021F36C2C4C227
:101EA400C1301103021F2EC2C5021F36900202E088
:101EB4007020E5C2F0E0FFC3900204E09F7480F854
:101EC400900203E06480985003122DB5900202E062
:101ED40004F0900204E024FFF0900203E034FFF0E9
:101EE40090020DE0FEA3E0240FF58274023EF58318
:101EF400E5C2F090020DE475F001121BA0FEE5F0BE
:101F040064404E700690020DF0A3F0900202E014BB
:101F1400F0700E900263E004F07006900262E00438
:101F2400F0D2C1800DC2C4301108C211D2C58002E2
:101F3400D21830181053C17F43C180C2C5C2C4C275
:071F4400C1C218C213C2C0A4
:101F4B00D007D006D000D0D0D082D083D0F0D0E054
:011F5B003253
:0531D200E5C15420FFDF
:0131D70022D5
:0731B80043C14053E6FE2273
:1020CA009002C3E0FFA3E0FCA3E0FDA3E0FBA3E0D2
:1020DA00FAA3E0F9900295E51AF0E51BA3F0900245
:0620EA00CBE0900297F02C
:1020F00090028FEFF0A3ECF0A3EDF0A3EBF0A3EAD6
:04210000F0A3E9F06F
:102104009002987403F0A374E8F0E5C120E5FBD2D3
:10211400C1C2C4D2C5E4FF900346F030C0FDE5C09F
:1021240054FE244070030221C724FE602424E2608C
:102134000924FE600524E20221CFC2C5EF60030238
:1021440021D590028FE025E044A0F5C27F0302214F
:10215400D5EFB4030A900290E0F5C27F058072EFD8
:10216400B4050B900290A3E0F5C27F068063EF6490
:1021740006703E900297E0900292700FE0FBA3E499
:1021840075F001121BB6A9F0FA8008E0FBA3E0FA8F
:10219400A3E0F9121B26F5C2900296E024FFF0900A
:1021A4000295E034FFF0E07002A3E070247F078022
:1021B40020EFB40706D2C47F098016900346740545
:1021C400F0800E9003467402F0800690034674017A
:1021D400F0EFB40904C2C08036900346E0FE640602
:1021E4006012EEB4021690029874FFF5F0121BA070
:1021F40045F06008D2C5E4900346F0FF900346E042
:102204006008C2C5D2C4C2C08005C2C002211FE595
:04221400C120E5FB05
:0122180022A3
:102219009002A5EFF0A3ECF0A3EDF0A3EBF0A3EA95
:04222900F0A3E9F045
:10222D009002AD7403F0A374E8F0E5C120E5FBD294
:10223D00C1C2C4D2C5E4FF900346F030C0FDE5C075
:10224D0054FE24C8700302230A24AE607A24CA7097
:10225D000302231224FE603824E2600924FE600587
:10226D0024E202231AC2C5EF700F9002A5E025E00B
:10227D0044A0F5C27F03022320EF64016003022313
:10228D00209002A5E025E044A1F5C27F04022320A1
:10229D00EFB4030A9002A6E0F5C27F058075EFB496
:1022AD00050B9002A6A3E0F5C27F068066EFB4068B
:1022BD0006D2C57F01805CEFB404047F0280549088
:1022CD0003467405F0804C9002A8E0FBA3E475F082
:1022DD0001121BB6A9F0FAE5C2121B6C9002ACE01C
:1022ED0024FFF09002ABE034FFF0E07002A3E07049
:1022FD00087F09C2C1D2C4801A7F0280169003469E
:10230D007406F0800E9003467402F080069003462A
:10231D007401F0EFB40904C2C08036900346E0FEAC
:10232D0064066012EEB402169002AD74FFF5F01261
:10233D001BA045F06008D2C5E4900346F0FF900362
:10234D0046E06008C2C5D2C4C2C08005C2C0022228
:06235D0048E5C120E5FB8C
:012363002257
:102364009002C3EFF09002C6EBF0A3EAF0A3E9F009
:082374009002C4ECF0A3EDF0AF
:10237C00751C00543FF51D543F605CC37440951DA3
:10238C00FFE4951CFE9002C9E0FCA3E0FDC39FECAA
:10239C009E50068C1A8D1B80048E1A8F1B1220CA1D
:1023AC00900346E060037F02229002C5E0251BF0FB
:1023BC009002C4E0351AF09002CBE0700B9002C78B
:1023CC00E51A851BF0121BA0C39002CAE0951BF006
:1023DC009002C9E0951AF09002C9E0F51AA3E0F555
:1023EC001BD3E51B9400E51A94004070E51B944048
:1023FC00E51A940050131220CA900346E060037F44
:10240C000222E4F51AF51B80D89002C3E0FFA3E08A
:10241C00FCA3E0FDA3E0FBA3E0FAA3E0F990029596
:10242C00E4F074401220E6900346E060037F022241
:10243C0074C0251BF51B74FF351AF51A9002C5E004
:10244C002440F09002C4E03400F09002CBE0709194
:0E245C009002C775F040121BA00223ED7F0016
:01246A00224F
:103033009002ABE4F0A304F0122219900346E0607F
:07304300037F01227F002240
:102F8500900345EBF07B017A0379459002C9E4F0A3
:0A2F9500A304F0E4A3F01223642269
:102E1C00C0079002EDE0FFA3E09002ABCFF0A3EF70
:102E2C00F0D007122219900346E060037F01227F45
:022E3C00002272
:102F9F00C0079002F5E0FFA3E09002C9CFF0A3EFC6
:0A2FAF00F0E4A3F0D007122364221F
:0E2C2600900314EBF0A3EAF0A3E9F0A3EDF0A5
:102C3400E4900319F0900314E0FBA3E0FAA3E0F995
:102C4400A3E090030AF0900318E090030BF0E4FF74
:102C5400122918EFB4FF0D900319E0FE04F0EEC33F
:062C6400940340D17E0044
:012C6A002247
:0B2CCC0090033DEBF0A3EAF0A3E9F059
:102CD7007E007F007D10121D9590033DE0FBA3E071
:102CE700FAA3E0F97D101218C8EF7002FF227F01E6
:012CF70022BA
:1029FB009002AF7422F0A3EFF0A37413F0121B2616
:102A0B009002B2F0900001121B3F9002B3F09000C5
:102A1B0002121B3F9002B4F0900003121B3F900276
:102A2B00B5F0900004121B3F9002B6F09000051217
:102A3B001B3F9002B7F0900006121B3F9002B8F0BC
:102A4B007B017A0279AFE4900318F07D0A022C2601
:102E3E0090032D7422F0A3EFF0A37403F0A374FF9C
:102E4E00F07B017A03792DE4900318F07D04022CB7
:012E5E00264D
:102E5F009003317422F0A3EFF0A3741CF0A374FF5E
:102E6F00F07B017A037931E4900318F07D04022C92
:012E7F00262C
:102EC100E4900335F0A3EFF0A3740AF0A3EFF07BD5
:0F2ED100017A037935E4900318F07D04022C2672
:102E8000A2AFE433FCC2AF758F0175B7A575B7F17A
:102E90008F828E83EDF0E4F58FAF04EF24FF92AFC5
:012EA000220F
:102EA100A2AFE433FDC2AF758F0375B7A575B7F156
:0F2EB1008F828E83E4F0F58FAF05EF24FF92AF91
:012EC00022EF
:102ABA00900339EEF0A3EFF0A3ECF0A3EDF0EB4AAC
:102ACA006039900339E0FEA3E0FFA3E0FCA3E0F540
:102ADA00828C83E0FD122E80EB1B70011A90033C5E
:102AEA00E004F0700690033BE004F090033AE0043F
:0C2AFA00F070CB900339E004F080C322A0
:0831B000E4900000F0A3F022FE
:102D2100900000E0FEA3E0FF122EA1900000E0FE63
:102D3100A3E0FF7C007D027B007A02122ABAE490B4
:062D41000000F0A3F022E7
:0A280500A90590031AEEF0A3EFF00E
:10280F00EE54FEFE900000E0FCA3E0FD7002EE6CC3
:10281F006057ED4C6003122D2190031AE0FEEE5429
:10282F00FEFE7F00900000F0A3EFF090031CEEF08F
:10283F00A3EFF0A37400F0A37402F07E0290031CC8
:10284F00E475F001121BB685F082F583E493FD90D9
:10285F00031EE475F001121BB685F082F583EDF0CF
:10286F00EF1F70011EEF4E70D490031AE0FCA3E02F
:10287F00FDEC5401FC74022DF58274003CF583E9E4
:01288F00F058
:012890002225
:102BE00090030DEEF0A3EFF0A3EBF0A3EAF0A3E95E
:102BF000F090031274FFF5F0121BB645F0602690BA
:102C0000030DE475F001121BB6AFF0FE90030FE068
:102C1000FBA3E475F001121BB6A9F0FA121B26FD06
:062C200012280580CC2201
:0B316A00C2A6D2A775380B7539B82239
:0B317500D2A6C2A775380B7539B8222E
:0713350090029AEFF0AB05F6
:10133C00C2AFC20CE0FF240AF8E6900324F0FD745F
:10134C00122BF8E6F9C39DFCE4940090029BF0A3E9
:10135C00CCF0300D4D90029BE0FCA3E0FDC3EC649F
:10136C00809480502E740E2FF8E670027603900253
:10137C009AE0FF240EF816E66003021411740E2F87
:10138C00F8760174122BF8E6FE740A2FF8A606D232
:10139C000C8072D3ED9404EC64809480405EC20D9A
:1013AC00804D90029BE0FEA3E0FFD39400EE64809E
:1013BC009480402E90029AE0240EF8E67002760398
:1013CC0090029AE0FD240EF816E67039740E2DF892
:1013DC00760174122BF8E6FC740A2DF8A604D20CD4
:1013EC008023C3EF94FCEE6480947F500FD20D9059
:1013FC00029AE0240AF8A601D20C800990029AE025
:10140C00240EF8E4F6E50945086003021729200CC0
:10141C000302172990029AE0FD2452F8E6FE74208C
:10142C002DF582E43403F583E0FDEDFFE4FCFD9043
:10143C00029D121D2090029BE0FEA3E0FFD39400BE
:10144C00EE64809480500302155DEE3395E0FDFC54
:10145C007810121D0D9002A1121D209002A1E0FC2B
:10146C00A3E0FDA3E0FEA3E0FFC006C007900324A9
:10147C00E0FFC374FF9FFFE49400AB07FAE4F9F8B4
:10148C00D007D006121C579002A1121D209002A169
:10149C00E0F8A3E0F9A3E0FAA3E0FBC00090029A05
:1014AC00E02452F8E6FFC374FF9FFFE49400FEE4CF
:1014BC00FCFDD000121BCC9002A1121D2090029AB0
:1014CC00E02452F8E6FF900324E0D39F9002A1E0C1
:1014DC00FCA3E0FDA3E0FEA3E0FFE440067B407A22
:1014EC000180037BC0FAF9F8121BCC9002A1121DEB
:1014FC002090029DE0F8A3E0F9A3E0FAA3E0FBC082
:10150C0000A3E0FCA3E0FDA3E0FEA3E0FF78101233
:10151C001CFAD000EB2FFFEA3EFEE93DFDE83CFC57
:10152C0090029D121D20E47FFF7EFFFDFC90029D2A
:10153C00E0F8A3E0F9A3E0FAA3E0FBD3121CE95016
:10154C000302166B90029D121D2C0000FFFF021669
:10155C006B90029BE0FEA3E0FFC3E49FFFE49EFEC2
:10156C003395E0FDFC7810121D0D9002A1121D2088
:10157C009002A1E0FCA3E0FDA3E0FEA3E0FFC00706
:10158C00900324E0FBE4FAF9F8D007121C57900200
:10159C00A1121D209002A1E0F8A3E0F9A3E0FAA3A8
:1015AC00E0FBC00090029AE02452F8E6FFE4FCFD58
:1015BC00FED000121BCC9002A1121D2090029AE0CA
:1015CC002452F8E6FF900324E0C39F9002A1E0FCB4
:1015DC00A3E0FDA3E0FEA3E0FFE450067B407A010C
:1015EC0080037BC0FAF9F8121BCC9002A1121D20CB
:1015FC0090029DE0FCA3E0FDA3E0FEA3E0FFC0048D
:10160C00C005C006C007A3E0FCA3E0FDA3E0FEA359
:10161C00E0FF7810121CFAA804A905AA06AB07D0A3
:10162C0007D006D005D004C3EF9BFFEE9AFEED99D0
:10163C00FDEC98FC90029D121D20E47FFF7EFFFDC7
:10164C00FC90029DE0F8A3E0F9A3E0FAA3E0FBD341
:10165C00121CE9400A90029D121D2C000000009003
:10166C00029DA3A3A3E0FF90029AE0FB2420F58245
:10167C00E43403F583EFF090029DE0FCA3E0FDA3BE
:10168C00E0FEA3E0FF7808121CFA90029D121D20C8
:10169C0074522BF8E6FFE4FCFDFE90029DE0F8A3EB
:1016AC00E0F9A3E0FAA3E0FBC3121CE9601490027A
:1016BC009DA3A3A3E0FF90029AE02452F8A6071280
:1016CC002FD2300D2A90029AE0FF240AF8E6FE246D
:1016DC0004FDE433FC74522FF8E6FFD39DEC6480D8
:1016EC00F87480984002801BEFC39E502980229092
:1016FC00029AE0FF240AF8E6FE74522FF8E6FFD3B4
:10170C009E400512316A8015EE24FCFEEFC39E50FC
:0F171C00051231758007D2A6D2A7122B06D2AFC5
:01172B00229B
:0B246B009002F7EBF0A3EAF0A3E9F009
:10247600900003121B3F9002FCF0E0FF540FA3F004
:10248600900006121B3F9002FEF0EF54F06490702D
:1024960055E060529002FDE030E30D200B0A123049
:1024A60060121A27D203D2059002FDE030E20D2019
:1024B6000B0A1231141231C6D204D2079002FDE083
:1024C60030E10D300B0A123060121A27D203D20502
:1024D6009002FDE030E073300B701231141231C6F9
:1024E600D204D20780649002FCE054F0FF6480605E
:1024F6000BEF649070309002FEE0702A9002FDE0CF
:10250600FF30E305200B02C203EF30E205200B0289
:10251600C204EF30E105300B02C203EF30E02B308E
:102526000B28C20480249002FCE054F0FFBFB01ACE
:102536009002F7E0FBA3E0FAA3E0F9900006121B75
:0C2546003FFF9002FAE4F0A3EFF07F00EA
:012552002266
:042E17004102E6008E
:0631D800E49002E6F02283
:0731BF009002E67401F0220A
:102891009003407404F0E4A3F0FFA3F01231B07E82
:1028A1003A7F017B017A037940900312E4F0A3049B
:1028B100F0122BE0E4FF74522FF8E4F60FEFB404AA
:1028C100F5E4F54FF550F551900341F0900341E0E7
:1028D100FFC3941E5029EF75F007A42402F582E48A
:1028E100343AAF82FE7B007A00794F900312E4F014
:1028F100A37407F0122BE0900341E004F080CD7E39
:102901003A7F007B017A037942900312E4F0A30439
:07291100F0122BE0022D2162
:102FD20020161530020D20B40D9002E6E07007D2E3
:092FE2000980031231E8D2162225
:10301B00903A00E493F46007A3E493640460031212
:08302B002891E49002DEF0227E
:102CF8009002DEE0FFC3941E501EEF75F007A42477
:102D080002F9743A35F0FA7BFF784F7C007D007E3B
:092D1800007F07121B00C2162205
:102C6B009002DEE0C3941E502A1231B09002DEE0D7
:102C7B0075F007A42402F582E4343AAF82FE7B00A0
:102C8B007A00794F900312E4F0A37407F0122BE053
:042C9B00122D2122B3
:0631DE00122C6BC2162248
:0526BE00900284EDF024
:1026C300900286E004F0900289EFF0A3EBF0900211
:1026D30084E0FF900289E0FED39F400302276FEE60
:1026E30075F007A42402F582E4343AAF8290028B9A
:1026F300F0A3EFF090028AE075F007A42402F582BC
:10270300E4343AAF8290028DF0A3EFF0E4900287B5
:10271300F0A3F090028DE475F001121BB6AFF0FE4A
:1027230090028BE0FCA3E0F5828C83E493FD1228F6
:102733000590028CE004F0700690028BE004F090A8
:102743000288E004F07006900287E004F0C3900270
:1027530088E09407900287E0940040B7122D2190FF
:0C2763000289E004F0A3E004F00226D19B
:01276F002247
:051F5C009002CCEDF045
:101F61009002D1EFF0A3EBF09002CCE0FF9002D110
:101F7100E0D39F40030220C9A3E075F007A4240227
:101F8100F582E4343AAF829002CDF0A3EFF0E49011
:101F910002D3F0A3F09002D3E0FEA3E0FFC39407C5
:101FA100EE940050389002CDE0FCA3E0F5828C83E2
:101FB100E493FD74DF2FF582E43402F583EDF090B4
:101FC10002CEE004F070069002CDE004F09002D45D
:101FD100E004F070C09002D3E004F080B89002D128
:101FE100E075F007A42402F582E4343AAF8290024E
:101FF100CFF0A3EFF09002D2E075F007A42402F530
:1020010082E4343AAF829002CDF0A3EFF0E4900283
:10201100D3F0A3F09002CDE475F001121BB6AFF03E
:10202100FE9002CFE0FCA3E0F5828C83E493FD12E5
:1020310028059002D0E004F070069002CFE004F091
:102041009002D4E004F070069002D3E004F0C39053
:1020510002D4E094079002D3E0940040B79002D1FB
:10206100E075F007A42402F582E4343AAF829002CD
:10207100CFF0A3EFF0E49002D3F0A3F09002D3E00D
:10208100FCA3E0FDC39407EC9400502C9002CFE434
:1020910075F001121BB6AFF0FE74DF2DF582E4344A
:1020A10002F583E0FD1228059002D4E004F070CC23
:1020B1009002D3E004F080C4122D219002D1E004FB
:0820C100F0A3E004F0021F6926
:0120C90022F4
:0B2553009002B9EFF0A3EDF0A3EBF055
:10255E00A2AFE433A3F0C2AF1231B89002BAE0FEDC
:10256E009002B9E0FDEDFF9002C1EEF0A3EFF0E4B2
:10257E009002BDF09002BBE0FF9002C1E0FCA3E030
:10258E00FD7B017A0279DF9002EDE4F0A37407F08F
:10259E00122E1C9002C2E02407F09002C1E034001B
:1025AE00F09002BDE075F007A42402F9743A35F0FC
:1025BE00FAA374FFF0A3EAF0A3E9F01231B090028F
:1025CE00BEA3E0FAA3E0AE02FF7B017A0279DF90B0
:1025DE000312E4F0A37407F0122BE0122D219002E7
:1025EE00BDE004F0E0C3941E408A900304E0FF12A5
:0A25FE00312E9002BCE024FF92AFE2
:0126080022AF
:0B2770009002D5EFF0A3EDF0A3EBF01A
:10277B00A2AFE433A3F0C2AF1231B89002D6E0FEA1
:10278B009002D5E0FDEDFF9002DAEEF0A3EFF0E45E
:10279B009002D9F09002D9E0FFC3941E504BEF7515
:1027AB00F007A42402F582E4343AAF82FE9002DCF7
:1027BB00F0FAA3EFF0FB9002D7E0FF9002DAE0FC17
:1027CB00A3E0FDA9037BFF9002F5E4F0A37407F0EF
:1027DB00122F9F9002DBE02407F09002DAE0340026
:1027EB00F09002D9E004F080AB900304E0FF1231CB
:0927FB002E9002D8E024FF92AFF9
:0128040022B1
:1008A7000133330131B601303A012EBD012D41012B
:1008B7002BC4012A480128CB01274F0125D2012447
:1008C700560122D901215D011FE0011E64011CE7C9
:1008D700011B6B0119EE0118720116F5011578015C
:1008E70013FC01127F011103010F86010E0A010C8F
:1008F7008D010B1101099401081801069B01051FC1
:100907000103A201050A0104F40104DF0104CA017D
:1009170004B50104A001048B0104760104600104FD
:100927004B01043601042101040C0103F70103E222
:100937000103CC0103B70103A201038D0103780171
:10094700036301034E01033801032301030E010270
:10095700F90102E40102CF0102BA0102A401028FE8
:1009670001027A01028801028101027A0102730100
:10097700026C01026501025E010257010250010289
:100987004901024201023B01023401022D01022604
:1009970001021F01021801021101020901020201ED
:1009A70001FB0101F40101ED0101E60101DF010194
:1009B700D80101D10101CA0101C30101BC0101B57F
:1009C7000101AE0101AB0101A101019701018D01F7
:1009D700018401017A01017001016601015C0101D5
:1009E7005201014801013F01013501012B0101219C
:1009F70001011701010D0101030100F90100F001D7
:100A070000E60100DC0100D20100C80100BE0100C0
:100A1700B40100AB0100A101009701008D01008323
:100A270001007901008001007D01007B0100780150
:100A3700007501007201006F01006D01006A01007D
:100A47006701006401006101005E01005C0100595B
:100A570001005601005301005001004E01004B01F7
:100A6700004801004501004201003F01003D01002F
:100A77003A01003701003401003101002F01002C39
:100A870001002901002B01002A010029010028018A
:100A97000027010026010025010024010023010091
:100AA7002201002102004002003E02003C02003AFF
:100AB700020038020036020034020032020030021F
:100AC700002E02002C03003F03003C030039030003
:100AD7003603003303003004003C040038040034BC
:100AE70005003D04003305003F05003D05003C05BA
:100AF700003A05003905003805003606003F0600B4
:100B07003E06003C06003A06003906003707003E5D
:100B170007003C07003A07003808003E08003C0879
:100B2700003A09003E09003C0A003F0A003D0B005D
:100B3700400B003C0C003F0C003B0D003C0E003D01
:100B47000F003D0E003C0F003F0F003D100040100E
:100B5700003E10003C11003F11003D12003F120003
:100B67003D13003E14004014003E15003F160040A0
:100B770016003D17003E18003E19003E1A003E1BA6
:100B8700003E1D00401E003F1F003E21003F230086
:100B97003F25003F27003F2A003F2D003F30003F01
:100BA70034003F30003F31004031004031004031D8
:100BB700004031003F31003F31003F31003F3100FD
:100BC7003F31003F320040320040320040320040A7
:100BD70032003F32003F32003F32003F32003F32A7
:100BE700003F3300403300403300403300403300C0
:100BF7003F33003F33003F33003F33003F33003F75
:100C070034004034004034004034003F34003F3467
:100C1700003F34003F34003F34003F35004035008B
:100C27004035004035003F35003F35003F35003F38
:100C370035003F360040360040360040360040362B
:100C4700003F36003F36003F36003F36003F370053
:100C57004037004037004037003F37003F37003FFD
:100C670037003F37003F38004038004038004038F1
:100C7700003F38003F38003F38003F38003F390019
:100C87004039004039004039003F39003F39003FC3
:100C970039003F3A00403A00403A00403A003F3AB4
:100CA700003F3A003F3A003F3B00403B00403B00DB
:100CB700403B00403B003F3B003F3B003F3C004088
:100CC7003C00403C00403C00403C003F3C003F3C77
:100CD700003F3D00403D00403D00403D003F3D009E
:100CE7003F3D003F3D003F3E00403E00403E00404C
:100CF7003E003F3E003F3E003F3F00403F00403F39
:100D070000403F003F3F003F3F003F400040400062
:100D17004040004040003F40003F40003F4100400E
:100D270041004041004041003F41003F41003F42F8
:100D3700004042004042004042003F42003F420024
:100D47003F43004043004043004043003F43003FD0
:100D570044004044004044004044003F44003F44B6
:100D6700003F45004045004045003F45003F4500E6
:100D77003F46004046004046004046003F46003F91
:100D870047004047004047003F47003F47003F4874
:100D9700004048004048003F48003F4900404900A4
:100DA7004049004049003F49003F4A00404A00404F
:100DB7004A00404A003F4B00404B00404B00404B2D
:100DC700003F4B003F4C00404C00404C003F4C0064
:100DD7003F4D00404D00404D00404D003F4E00400C
:100DE7004E00404E00404E003F4F00404F00404FE6
:100DF70000404F003F50004050004050004050001E
:100E07003F51004051004051003F51003F520040C8
:100E170052004052003F530040530040530040539C
:100E2700003F54004054004054003F54003F5500D9
:100E37004055004055003F56004056004056003F81
:100E470057004057004057003F57003F5800405851
:100E5700004058003F59004059004059003F5A0090
:100E6700405A00405A003F5B00405B00405B003F38
:100E77005C00405C00405C003F5D00405D00405D01
:100E8700003F5E00405E00405F00405F00405F0043
:100E97003F60004060004060003F610040610040EB
:030EA700620040A6
:03000000020800F3
:03000300021A03DB
:03000B00021A06D0
:03001300021A09C5
:03001B00021A0CBA
:03002300021A0FAF
:03002B00021A12A4
:03003300021A1599
:03003B00021A188E
:03004300021A1B83
:03004B00021A1E78
:03005300021A216D
:03005B00021A2462
:03006300021A2757
:03006B00021A2A4C
:03007300021A2D41
:10080000E4F5D9E5EF7480F5FF7402F5EF787FE445
:10081000F6D8FD9000007F007E04E4F0A3DFFCDE4C
:07082000FA75815502086220
:10082700020EAAE493A3F8E493A34003F68001F22F
:1008370008DFF48029E493A3F85407240CC8C333D2
:10084700C4540F4420C8834004F456800146F6DFA1
:10085700E4800B0102040810204080902DFAE47E0A
:10086700019360BCA3FF543F30E509541FFEE49396
:10087700A360010ECF54C025E060A840B8E493A35D
:10088700FAE493A3F8E493A3C8C582C8CAC583CA88
:10089700F0A3C8C582C8CAC583CADFE9DEE780BE40
:012E1B0000B6
:101A3000E709F608DFFA8046E709F208DFFA803E98
:101A400088828C83E709F0A3DFFA8032E309F60885
:101A5000DFFA8078E309F208DFFA807088828C83ED
:101A6000E309F0A3DFFA806489828A83E0A3F608A1
:101A7000DFFA805889828A83E0A3F208DFFA804C7B
:101A800080D280FA80C680D4806980F28033801052
:101A900080A680EA809A80A880DA80E280CA8033BB
:101AA00089828A83ECFAE493A3C8C582C8CCC58333
:101AB000CCF0A3C8C582C8CCC583CCDFE9DEE78003
:101AC0000D89828A83E493A3F608DFF9ECFAA9F082
:101AD000EDFB2289828A83ECFAE0A3C8C582C8CCD8
:101AE000C583CCF0A3C8C582C8CCC583CCDFEADEF1
:101AF000E880DB89828A83E493A3F208DFF980CC53
:101B000088F0EF60010E4E60C388F0ED2402B4044B
:101B10000050B9F582EB2402B4040050AF232345F2
:061B20008223901A80737D
:101B2600BB010689828A83E0225002E722BBFE02BD
:091B3600E32289828A83E49322F0
:101B3F00BB010CE58229F582E5833AF583E022505B
:101B4F0006E92582F8E622BBFE06E92582F8E222A5
:0D1B5F00E58229F582E5833AF583E49322BF
:101B6C00BB010689828A83F0225002F722BBFE0158
:021B7C00F32252
:101B7E00F8BB010DE58229F582E5833AF583E8F09D
:101B8E00225006E92582C8F622BBFE05E92582C849
:021B9E00F22231
:101BA000C5F0F8A3E028F0C5F0F8E58215827002D0
:061BB0001583E038F0226D
:101BB600A3F8E0C5F025F0F0E582158270021583E2
:061BC600E0C838F0E8223F
:101BCC00E88FF0A4CC8BF0A42CFCE98EF0A42CFCB8
:101BDC008AF0EDA42CFCEA8EF0A4CDA8F08BF0A436
:101BEC002DCC3825F0FDE98FF0A42CCD35F0FCEB95
:101BFC008EF0A4FEA9F0EB8FF0A4CFC5F02ECD395A
:0F1C0C00FEE43CFCEAA42DCE35F0FDE43CFC22C6
:101C1B0075F008758200EF2FFFEE33FECD33CDCC80
:101C2B0033CCC58233C5829BED9AEC99E582984003
:101C3B000CF582EE9BFEED9AFDEC99FC0FD5F0D6E0
:101C4B00E4CEFBE4CDFAE4CCF9A88222B800C1B90A
:101C5B000059BA002DEC8BF084CFCECDFCE5F0CB48
:101C6B00F97818EF2FFFEE33FEED33FDEC33FCEB81
:101C7B0033FB10D703994004EB99FB0FD8E5E4F93C
:101C8B00FA227818EF2FFFEE33FEED33FDEC33FC29
:101C9B00C933C910D7059BE99A4007EC9BFCE99A1D
:101CAB00F90FD8E0E4C9FAE4CCFB2275F010EF2F62
:101CBB00FFEE33FEED33FDCC33CCC833C810D70762
:101CCB009BEC9AE899400AED9BFDEC9AFCE899F89D
:0E1CDB000FD5F0DAE4CDFBE4CCFAE4C8F92230
:101CE900EB9FF5F0EA9E42F0E99D42F0E89C45F051
:011CF90022C8
:101CFA00E8600FECC313FCED13FDEE13FEEF13FFC8
:031D0A00D8F122EB
:101D0D00E8600FEFC333FFEE33FEED33FDEC33FC34
:031D1D00D8F122D8
:0C1D2000ECF0A3EDF0A3EEF0A3EFF02236
:101D2C00A8828583F0D083D082121D43121D4312EA
:101D3C001D43121D43E473E493A3C583C5F0C5830F
:101D4C00C8C582C8F0A3C583C5F0C583C8C582C801
:011D5C002264
:0C1D5D00A42582F582E5F03583F5832291
:101D6900D083D082F8E4937012740193700DA3A309
:101D790093F8740193F5828883E47374029368601D
:061D8900EFA3A3A380DF1D
:061D8F008A838982E473DF
:101D9500EF4E6012EF60010EEDBB010B89828A8365
:101DA500F0A3DFFCDEFA2289F05007F709DFFCA972
:0C1DB500F022BBFEFCF309DFFCA9F022C9
:00000001FF
